:100000000C9488000C9429120C94A5000C94A50063
:100010000C94A5000C94A5000C94A5000C94A500CC
:100020000C94A5000C94A5000C94A5000C94A500BC
:100030000C94A5000C94A5000C94A5000C94A500AC
:100040000C94A5000C94A5000C94A5000C94A5009C
:100050000C94A5000C94A5000C94A5000C94A5008C
:100060000C94A5000C94A5001201100100000008DA
:100070005E040202000100000001090220000101EB
:100080000080320904000002584200000705820384
:1000900020000407050203080004FF0004FF060710
:1000A00005FF020103FFFFFFFFFFFF00020104FF46
:1000B00003FF0607FFFF05040309042A03770077FF
:1000C0000077002E006200720075006E006F0066FF
:1000D000007200650069007400610073002E006307
:1000E000006F006D002A03550053004200200052AB
:1000F000006500740072006F005000610064002011
:10010000004100640061007000740065007200002E
:1001100011241FBECFEFD4E0DEBFCDBF11E0A0E0C1
:10012000B1E0E6E6F7E202C005900D92A230B10719
:10013000D9F711E0A2E0B1E001C01D92A13DB107E5
:10014000E1F70E9472050C94B1130C9400000F9318
:100150001F93FF93EF93BF93AF93F92FE82F09E01D
:100160000093580100E20093590100E000935A0106
:1001700001E000935B0101E000935C0100E000936B
:100180005D0100935E0100935F0109E2009360014D
:1001900007D0BF91AF91EF91FF911F910F910895FB
:1001A000A1E0B8E509E02D980000000000002C98BF
:1001B0000000000000002C9A000000002C980000B5
:1001C000000000002C9A0000000000002C980000A5
:1001D000000000002C9A0000000000002C98000095
:1001E000000000002C9A00000000000000002D9A82
:1001F0001D9117FD2C9A17FF2C982D9800000000D8
:100200002C9A16FD2D9A16FF2D982C9A00000000AE
:100210002D9A15FD2C9A15FF2C982D9A00000000A0
:100220002C9A14FD2D9A14FF2D982C9A0000000092
:100230002D9A15FD2C9A15FF2C982D9A0000000080
:100240002C9A14FD2D9A14FF2D982C9A0000000072
:100250002D9A15FD2C9A15FF2C982D9A0000000060
:100260002C9A14FD2D9A14FF2D982C9A0000000052
:100270002D9A0A952D9A2C9A0895F92FE82FCF934D
:10028000DF93D72FC62F21E030E0E20FF31F2227A4
:10029000332744275527662777278827992790E013
:1002A00099D0B6D082D0292F80D0392F7ED0492F37
:1002B000253031F02930A1F180E0DF91CF91089510
:1002C000BFEFBA95F1F7B8ECBA95F1F791E082D0AB
:1002D0009FD06BD0292F69D0392F67D0492F65D097
:1002E000592F4083518340E050E027FD426026FDB6
:1002F000416025FD546024FD52602F7035FD40643F
:1003000034FD406833FD486032FD446031FD40619A
:1003100030FD406245835683822FDF91CF9108954F
:10032000B4E6BA95F1F790E455D093E053D092E05B
:1003300051D06ED03AD0292F38D0392F36D0492F0E
:1003400034D0592F32D0692F30D0792F2ED0892F29
:100350002CD0405850584083518360587058628365
:10036000738340E050E020FD426021FD416022FDAA
:10037000486023FD446024FD526034FD546035FD27
:10038000406836FD406436FF8C8335FF9D8345838E
:1003900056833F70232F3E7F31FD31603D7F20FD2E
:1003A0003260832FDF91CF91089590E0B4E1A8E00F
:1003B000BA9579F01899FCCFB9E0BA95F1F7990F91
:1003C00018999160B4E1BA9521F0189BFCCFAA95D9
:1003D00079F70895A8E097FD0DC0209ABDE0BA9581
:1003E000F1F700002098B3E0BA95F1F7990FAA95BC
:1003F00091F70895209AB3E0BA95F1F70000000054
:100400002098BDE0BA95F1F7990FAA9521F70895C4
:10041000209AB3E0BA95F1F7000000002098089503
:10042000A8950895FC01808190E0807690708032DC
:10043000910559F481818130E1F483E391E0909357
:1004400093018093920184E108958034910589F4A9
:100450008181863071F481E090E090930301809374
:10046000020187E491E0909393018093920180E1EF
:10047000089580E00895809102019091030108950C
:10048000CF93DF938091AE0186FD07C0CEEAD1E025
:100490000E94B710888186FFFBCF83E391E064E17F
:1004A0000E940612DF91CF910895E3E3F1E084E228
:1004B000DF011D928A95E9F794E1918380E1848BB5
:1004C00082E4858B168A81E0878B808F82E0818F22
:1004D000928F86E0838F7C962FEF87E591E02193C2
:1004E000E817F907E1F708950F931F938C010E9415
:1004F0005502012B61F02FE088E190E00FB6F894EF
:10050000A895809360000FBE2093600008C088E12A
:100510000FB6F89480936000109260000FBE0E94A6
:10052000A010F894EAE2F0E080818260808380810C
:100530008660808326EF39E040E951E0CA010197E7
:10054000F1F721503040D1F7EAE2F0E080818D7F71
:1005500080838081897F808378941F910F91089593
:100560002F923F924F925F926F927F928F929F92C3
:10057000AF92BF92CF92DF92EF92FF920F931F93B1
:10058000DF93CF93CDB7DEB73B014C0119012A01B0
:100590006D897E898F89988D6A197B098C099D09DF
:1005A000621A730A840A950AA40193010E945513E2
:1005B000E218F30804091509A80197010E947413B1
:1005C0002A0D3B1D4C1D5D1D622F732F842F952F0F
:1005D000CF91DF911F910F91FF90EF90DF90CF901F
:1005E000BF90AF909F908F907F906F905F904F9053
:1005F0003F902F9008951AB889EF8BB914B88FE304
:1006000085B917B888B908952F923F924F925F929B
:100610006F927F928F929F92AF92BF92CF92DF9212
:10062000EF92FF920F931F93CF93DF93EC01DB01C7
:100630008D8180FF06C0E5E3F1E0808181608083E9
:1006400005C0E5E3F1E080818E7F80838D8182FFAC
:1006500006C0E5E3F1E080818260808305C0E5E3C8
:10066000F1E080818D7F80838D8183FF06C0E5E38B
:10067000F1E080818460808305C0E5E3F1E0808162
:100680008B7F80838D8181FF06C0E5E3F1E080816F
:100690008860808305C0E5E3F1E08081877F808307
:1006A0008F8181FF06C0E5E3F1E080818061808376
:1006B00005C0E5E3F1E080818F7E80838F8180FF3C
:1006C00006C0E5E3F1E080818062808305C0E5E358
:1006D000F1E080818F7D80838F8182FF06C0E5E31A
:1006E000F1E080818064808305C0E5E3F1E08081F2
:1006F0008F7B80838F8183FF06C0E5E3F1E08081FB
:100700008068808305C0E5E3F1E080818F77808396
:100710008E8180FD02C080E001C08FEF80933701A1
:100720008E8181FD02C080E001C08FEF809338018F
:100730008E8182FD02C080E001C08FEF809339017D
:100740008E8183FD02C080E001C08FEF80933A016B
:100750008E8186FD02C080E001C08FEF80933D0155
:100760008E8187FD02C080E001C08FEF80933E0143
:100770008E8185FD02C080E001C08FEF80933B0138
:100780008E8184FD02C080E001C08FEF80933C0128
:100790008C91882311F08093370112968C911297D7
:1007A000882311F08093390113968C911397882335
:1007B00011F080933A0111968C911197882311F0D2
:1007C0008093380114968C911497882311F08093AC
:1007D0003D0115968C911597882311F080933E0169
:1007E00016968C911697882311F080933B011796EB
:1007F0006C91662311F060933C0100D000D0EDB7FE
:10080000FEB73196698170E080E090E02FEF3FE71E
:1008100040E050E0208331834283538320E83FEF60
:100820004FEF5FEF0F2EFFE7EF2EF0E0FF2EF0E02F
:100830000F2FF0E01F2FF02D0F2EF0E0AF2EF0E87D
:10084000BF2EFFEFCF2EFFEFDF2EF02D0E94B00264
:100850000F2EFFE36F2EF1E07F2EF02DF301619359
:1008600071934F01EDB7FEB731966A8170E080E079
:1008700090E00F2EF0E02F2EF0E83F2EFFEF4F2EEE
:10088000FFEF5F2EF02D208231824282538220E8DA
:100890003FEF4FEF5FEF0F2EFFEFAF2EFFE7BF2EC3
:1008A000F0E0CF2EF0E0DF2EF02D0E94B002F40138
:1008B00071836083EDB7FEB731966B8170E080E0A5
:1008C00090E0A082B182C282D38220E83FEF4FEF56
:1008D0005FEF0F2EF0E0AF2EF0E8BF2EFFEFCF2E30
:1008E000FFEFDF2EF02D0E94B002F30134967183EA
:1008F0006083EDB7FEB731966C8170E080E090E0E8
:10090000208231824282538220E83FEF4FEF5FEF37
:100910000F2EFFEFAF2EFFE7BF2EF0E0CF2EF0E05F
:10092000DF2EF02D0E94B0020F900F900F900F90CD
:1009300026E030E0620E731EF30171836083DF9165
:10094000CF911F910F91FF90EF90DF90CF90BF90CC
:10095000AF909F908F907F906F905F904F903F905F
:100960002F900895682FF894A4E0B1E0E9E1F1E058
:1009700088E001900D928150E1F760930401ACE0B2
:10098000B1E0E1E2F1E085E001900D928150E1F704
:1009900060930C01A1E1B1E0E6E2F1E088E00190B2
:1009A0000D928150E1F735995BC0349952C086B100
:1009B00090E08E7190708430910521F18530910521
:1009C00034F4009771F0029709F056C00FC08830D8
:1009D000910511F18A309105D1F0069709F04CC0CC
:1009E0000CC084E091E00E94610E5EC084E091E062
:1009F00061E171E00E94CF0C57C084E091E00E9459
:100A0000AD0852C084E091E00E94870938C084E0BC
:100A100091E00E94400848C083B190E086709070D9
:100A20008230910589F08630910521F0892B39F0CB
:100A300081E023C084E091E00E94940735C084E007
:100A400091E00E94260730C084E091E00E94B30943
:100A50002BC0339914C084E091E00E941C1024C084
:100A6000339905C084E091E00E94E4051DC084E054
:100A700091E00E94D00A03C080E08823A9F489B1E4
:100A8000897071F44C9B07C084E091E061E171E0F2
:100A90000E949D0509C084E091E00E947D0B04C086
:100AA00084E091E00E94000AE8E6F0E080818E7F19
:100AB000808378940895CF93DF9381E090E00E9443
:100AC0007402C0E4DCE907C00E941002CE01019765
:100AD000F1F70E9440020E943B02892BA9F3DF91AB
:100AE000CF9108950F931F93CF93DF930E94FB0242
:100AF0000E945B0581E00E94B20404E011E0C1E1C4
:100B0000D1E00E94100281E00E94B204C801BE013F
:100B10000E9404030E944002F4CFE4E2F0E020814E
:100B2000277F2083208120632083E5E2F0E020817D
:100B3000286320830E94A70008950F931F93CF93EB
:100B4000DF93EC018B01E5E2F0E080818E7F808312
:100B5000E4E2F0E080818E7F8083EBE2F0E0808150
:100B60008F778083EAE2F0E0808180688083CE0125
:100B70000E943D01282F83FF03C08D8181608D83FA
:100B800022FF03C08D8184608D8321FF03C08D818E
:100B900088608D8320FF03C08D8182608D83F80182
:100BA0008481833208F41482F8018581833208F449
:100BB00015828A8181958A838C8181958C83DF91CE
:100BC000CF911F910F910895DC01EAE2F0E080815E
:100BD0008E7E8083EBE2F0E0808181618083E4E2BD
:100BE000F0E080818863808380818D7F8083E5E26F
:100BF000F0E0808182608083E7E2F0E08081807EA7
:100C00008083E8E2F0E080818F618083489B0BC0A5
:100C1000E4E2F0E0808184608083E5E2F0E08081BE
:100C2000837C808314C0E4E2F0E080818B7F80834A
:100C3000E5E2F0E080818C638083E7E2F0E0808190
:100C40008E7F8083E8E2F0E080818160808387E1AD
:100C500080937E00EAE7F0E085E0808384E680937D
:100C60007C00808180688083808186FDFDCF61303B
:100C700009F5EAE7F0E0808180648083808186FD69
:100C8000FDCF909179008FE7891B12968C93129774
:100C900082E680937C00EAE7F0E0808180648083D4
:100CA000808186FDFDCF909179008FE7891B119699
:100CB0008C931197E9E2F0E0808110927A00109213
:100CC0007E00808180FF17C04C9909C0613039F4E3
:100CD00016968C911697816016968C931697199993
:100CE00098C0623009F095C016968C911697816075
:100CF00016968C930895E5E2F0E08081877F8083EB
:100D000085E08A95F1F7309907C016968C91169771
:100D1000826016968C9316971A9907C016968C9136
:100D20001697806116968C931697199907C0169698
:100D30008C911697806816968C9316974C9907C0DD
:100D400017968C911797846017968C931797E5E206
:100D5000F0E080818860808380818F7E808385E061
:100D60008A95F1F7309907C016968C911697846092
:100D700016968C9316971A9907C016968C9116970B
:100D8000806216968C931697199907C017968C91C6
:100D90001797816017968C9317974C9907C01696F2
:100DA0008C911697816016968C931697E5E2F0E089
:100DB00080818061808380818F7D808385E08A95BA
:100DC000F1F7309907C016968C91169788601696A1
:100DD0008C9316971A9907C016968C911697806473
:100DE00016968C931697199907C017968C9117979A
:100DF000826017968C9317974C9906C017968C9122
:100E00001797886017968C93E5E2F0E08081806206
:100E10008083089590E020E0A3E2B0E0EBE2F0E010
:100E200035E1220F8C9180FD216080818F77808356
:100E3000832F8A95F1F7808180688083832F8A953C
:100E4000F1F79F5F983069F7822F0895CF93DF9372
:100E5000EC01ABE2B0E08C91886F8C938C918E7F2B
:100E60008C93EAE2F0E08081896C808380818F7CC2
:100E70008083E4E2F0E080818E7F8083E5E2F0E031
:100E80008081816080838C918F7B8C930E940A0784
:100E9000282F30E0C901807F90708034910509F0DF
:100EA00040C020FF03C08D8188608D8321FF03C077
:100EB0008D8182608D8322FF03C08D8181608D834F
:100EC00023FF03C08D8184608D830E940A07282F31
:100ED000982F81FF03C08E8180648E8392FF03C0B0
:100EE0008E8180688E8393FF03C08F8181608F83A2
:100EF00094FF03C08F8182608F8395FF03C08E8132
:100F000084608E8396FF03C08E8182608E8322234D
:100F10001CF48E8181608E83EBE2F0E0808180643E
:100F20008083DF91CF910895DC01EAE2F0E08081D7
:100F300086708083EBE2F0E08081896F8083E4E259
:100F4000F0E08081807C8083E5E2F0E080818F6347
:100F50008083E9E2F0E08081982F9170808183FDA9
:100F6000926080912F01981709F466C09130F1F0DA
:100F7000913038F0923009F441C0933009F051C0FB
:100F800029C0813041F415968C9115978260159691
:100F90008C93159746C0823009F043C015968C910A
:100FA0001597886015968C9315973BC0833041F454
:100FB00015968C911597826015968C93159731C074
:100FC000882379F515968C911597886015968C93E2
:100FD000159727C0823041F415968C911597826041
:100FE00015968C9315971DC08130D9F415968C9168
:100FF0001597886015968C93159713C0882341F434
:1010000015968C911597826015968C93159709C04B
:10101000833039F415968C911597886015968C93CA
:10102000159790932F0183E080932E0115968C9154
:101030001597809330010CC080912E01882341F0D8
:10104000815080932E018091300115968C931597D5
:101050004E9906C016968C911697816016968C93C1
:101060000895EBE2F0E080818F7E80838CE291E056
:101070000197F1F789B19081906190838170089513
:10108000CF93DF93EC01E4E2F0E08081837C808306
:10109000808182608083A5E2B0E08C918E638C9326
:1010A000EAE2F0E080818E7F8083808180618083AE
:1010B000EBE2F0E08081816180838C918D7F8C9365
:1010C0001D9903C08D8181608D831C9903C08D8122
:1010D00084608D831B9903C08D8188608D831A99EC
:1010E00003C08D8182608D830E943108882319F4AA
:1010F0008E8182608E830E943108882319F48E814C
:1011000081608E830E943108882319F48E81886063
:101110008E830E943108882319F48E8184608E8327
:101120000E943108882319F48E8180688E830E9482
:101130003108882319F48E8180648E830E943108DF
:10114000882319F48F8182608F83E5E2F0E080814B
:1011500082608083DF91CF910895CF93DF93DC018C
:10116000E4E2F0E08081837C808380818260808300
:10117000E5E2F0E080818E638083EAE2F0E0808146
:1011800080618083EBE2F0E080818F7E808392E05B
:101190002BE230E0E3E2F0E045E250E0E901888153
:1011A0008F7E88830000000080818C7309F457C013
:1011B000808185FD07C015968C91159781601596E5
:1011C0008C931597808184FD07C015968C91159797
:1011D000826015968C931597808183FD07C01596C4
:1011E0008C911597846015968C931597808182FD5C
:1011F00007C015968C911597886015968C93159756
:10120000EA0188818D7F888300000000808185FD50
:1012100007C016968C911697826016968C93169737
:10122000808184FD07C016968C9116978160169672
:101230008C931697808183FD07C017968C91179722
:10124000816017968C931797808182FD36C0179620
:101250008C911797826017968C9317972EC0EA018E
:1012600088818D7F888300000000808185FD07C014
:1012700016968C911697846016968C93169780819B
:1012800084FD07C016968C911697886016968C93ED
:101290001697808183FD07C016968C9116978064FF
:1012A00016968C931697808182FD07C016968C91B6
:1012B0001697806816968C931697E901888180614D
:1012C0008883EA01888182608883915009F066CF23
:1012D000DF91CF91089590E020E0E5E2F0E03AE67A
:1012E000A3E2B0E080818B7F8083832F8A95F1F722
:1012F00026958C9185FD2068808184608083832F72
:101300008A95F1F79F5F983069F7822F0895EF92E1
:10131000FF920F931F937C0105E210E0F80180819A
:101320008C7E8083808184628083E4E2F0E080812F
:101330008F7D808380818C618083F80180818860CB
:10134000808388EC90E00197F1F70E946B09F80127
:101350008081877F80838AEAF70187831F910F91BD
:10136000FF90EF900895DC01EAE2F0E08081867062
:101370008083EBE2F0E08081896F8083E4E2F0E03B
:1013800080818E7F8083E5E2F0E0808181608083D0
:101390004E990CC016968C911697816016968C9378
:1013A000169704C09F5F9B3F21F4089590E0E3E20D
:1013B000F0E0808180FDF6CF89B1982F892F80954C
:1013C000282F217093FF226094FF246095FF2860EE
:1013D00090E0E3E2F0E003C09F5F9B3F81F08081FB
:1013E00080FFFACF89B180FF206183FF206284FFF4
:1013F000206485FF20688FE7821B11968C930895E7
:10140000DC01EAE2F0E08081867880838081806878
:101410008083EBE2F0E080818F7780838081896731
:101420008083E4E2F0E080818E7F8083E5E2F0E07B
:101430008081816080838AE48A95F1F789B1807325
:1014400011F090E015C04E9907C016968C91169732
:10145000816016968C931697189B02C091E008C085
:1014600017968C911797826017968C93179791E037
:10147000EBE2F0E08081806880838AE48A95F1F76E
:10148000489907C015968C911597816015968C9395
:1014900015974B9907C015968C91159784601596F2
:1014A0008C9315974C9907C015968C911597886069
:1014B00015968C9315974D9907C015968C91159795
:1014C000826015968C931597992391F44E9907C0D5
:1014D00016968C911697816016968C93169718998C
:1014E00059C016968C911697826016968C9352C0AE
:1014F0004E9907C016968C911697826016968C931B
:101500001697189907C016968C91169784601696B0
:101510008C931697EBE2F0E080818F7780839AE4DA
:10152000892F8A95F1F7808180688083892F8A9539
:10153000F1F780818F7780839A95F1F789B189736C
:1015400049F58081806880838AE48A95F1F748991B
:1015500007C016968C911697806816968C931697EE
:101560004B9907C016968C911697806416968C93AB
:1015700016974C9907C016968C9116978860169608
:101580008C9316974D9906C017968C91179781608A
:1015900017968C93EBE2F0E0808180688083089559
:1015A000DC01E4E2F0E08081817C8083E5E2F0E030
:1015B00080818E638083E7E2F0E08081807C80839D
:1015C000E8E2F0E080818F638083EAE2F0E08081EE
:1015D0008E7E8083EBE2F0E08081816180831D99C3
:1015E00007C017968C911797816017968C93179761
:1015F0001C9907C016968C911697886016968C9346
:1016000016971B9907C016968C91169782601696AE
:101610008C9316971A9907C015968C91159782602E
:1016200015968C931597199907C015968C91159757
:10163000846015968C931597329907C017968C91F4
:101640001797826017968C931797319907C0169653
:101650008C911697846016968C931697309906C0D5
:1016600016968C911697816016968C930895282F64
:10167000269511F437E009C037E0982F990F822F93
:101680008170892B31502695C1F790E002C0880FF8
:10169000991F3A95E2F7089589B1E5E2F0E090816B
:1016A0009E7F908320E8922F9A95F1F79081916028
:1016B00090832A95F1F78295869587708095817041
:1016C000089520E090E0A9E2B0E0E5E2F0E030E843
:1016D00026958C9185FF206880818E7F8083832F63
:1016E0008A95F1F7808181608083832F8A95F1F755
:1016F0009F5F983069F7822F08950F931F93CF93C0
:10170000DF93EC01EAE2F0E080818F7D8083ABE241
:10171000B0E08C9180628C938081806880838C9112
:1017200080688C93E4E2F0E0808181608083E5E270
:10173000F0E080818160808380EC90E00197F1F798
:101740008C918F778C9380E88A95F1F70E94610BDA
:10175000182F0E94610B082F0E94610B982F1123F4
:101760001CF48D8182608D83212F30E016FF03C031
:101770008D8188608D8325FF03C08D8184608D837A
:1017800024FF03C08D8181608D83F901E870F070C2
:1017900023FF03C08F8182608F83B90164707070F2
:1017A00022FF03C08F8181608F83892F8F708830E3
:1017B00009F05AC0812F82958F70982F80FF03C047
:1017C0008D8181608D8391FF03C08D8184608D83C5
:1017D00092FF03C08D8188608D8393FF03C08D814C
:1017E00082608D83802F8095482F4F70483008F09D
:1017F0004051842F90E0880F991F880F991F909572
:1018000081959F4F8A83802F90E080959095807F6F
:1018100090709595879595958795959587959595CC
:101820008795482F883008F04051842F90E0880F2A
:10183000991F880F991F909581959F4F8983EF2B52
:1018400019F08F8182608F83672B19F08F818160FF
:101850008F8321FF03C08E8181608E8320FF6CC047
:101860008E8182608E8368C0402F50E0CA01807CE8
:101870009070803C9105D1F50F3F21F081E080937D
:1018800031010FC080913101882359F421FF03C039
:101890008E8181608E8320FF4FC08E8182608E8317
:1018A0004BC020FF02C08FE78C8321FF02C080E87D
:1018B0008B8340FF02C08FE78B8341FF02C080E82B
:1018C0008C8342FF03C08E8180648E8343FF03C0FC
:1018D0008E8180688E8344FF03C08E8181608E83F9
:1018E00045FF2AC08E8182608E8326C0802F807F34
:1018F00009F51092310121FF03C08E8184608E832F
:1019000020FF03C08E8181608E8340FF03C08E81E3
:1019100082608E8341FF03C08E8188608E8342FF88
:1019200003C08E8180648E8343FF06C08E818068F1
:101930008E8302C010923101DF91CF911F910F91E0
:101940000895382F80E18A95F1F720E090E0E5E2F4
:10195000F0E040E4A3E2B0E030FF04C080818061A9
:10196000808303C080818F7E808380818B7F808392
:10197000842F8A95F1F726958081846080838C91ED
:1019800085FD2068842F8A95F1F79F5F983011F0CC
:101990003695E2CF80E18A95F1F7822F0895AF92D4
:1019A000BF92DF92EF92FF920F931F93CF93DF933B
:1019B000EC015B01E4E2F0E080818D7D8083808139
:1019C0008C618083E5E2F0E080818E63808380819A
:1019D000877F808380E18A95F1F781E00E94A10CE6
:1019E00082E40E94A10C182F00E0813409F401E088
:1019F000DD24133711F4DD24D394EE24FF241937AA
:101A000019F4EE24FF24E39480E090E0133511F400
:101A100081E090E09701282B392B802F8D2990E0D1
:101A2000282B392B232B09F4BDC08FEF0E94A10C6A
:101A30008FEF0E94A10C282F982F80FD03C08F816B
:101A400081608F8393FD03C08F8182608F83002329
:101A5000A9F094FD03C08D8181608D8396FD03C044
:101A60008D8184608D8322231CF08D8188608D831D
:101A700095FD16C08D8182608D8312C0DD2081F0BE
:101A800091FD03C08F8184608F8392FD03C08F819D
:101A900088608F83822F82958F7080958F708D8361
:101AA0008FEF0E94A10C282F982F80FD03C08E81FC
:101AB00080618E8391FD03C08E8180628E8392FD52
:101AC00003C08E8180648E8393FD03C08E81806805
:101AD0008E8394FD03C08E8188608E8395FD03C044
:101AE0008E8182608E8396FD03C08E8181608E839D
:101AF00022231CF08E8184608E8380E0133509F4EC
:101B000081E08D2990E08E299F29892BA1F08FEF0C
:101B10000E94A10C80588B838FEF0E94A10C8058EB
:101B20008C838FEF0E94A10C805889838FEF0E94D5
:101B3000A10C80588A831937A9F58FEF0E94A10C58
:101B40008FEF0E94A10C8FEF0E94A10C8FEF0E94DB
:101B5000A10C8FEF0E94A10CF50183838FEF0E94EF
:101B6000A10CF50181838FEF0E94A10CF501808308
:101B70008FEF0E94A10CF50182838FEF0E94A10CD0
:101B8000F50184838FEF0E94A10CF50185838FEF0F
:101B90000E94A10CF50187838FEF0E94A10CF50133
:101BA00086833BC01332C9F58FEF0E94A10C8FEFE3
:101BB0000E94A10C982F83FD03C08F8182608F83C8
:101BC000892F82958F7080958F708D838FEF0E9403
:101BD000A10C282F83FD03C08E8180688E8324FD95
:101BE00003C08E8188608E8325FD03C08E81826054
:101BF0008E838FEF0E94A10C805889838FEF0E9403
:101C0000A10CF50180838FEF0E94A10CF501828366
:101C10008FEF0E94A10CF5018483E5E2F0E0808162
:101C20008860808380E18A95F1F7DF91CF911F91E1
:101C30000F91FF90EF90DF90BF90AF900895EF92DB
:101C4000FF920F931F93CF93DF937C01E5E2F0E0C7
:101C50008081877F8083062F10E01016110664F4C0
:101C6000C0E0D0E0F701EC0FFD1F80810E94A10CC5
:101C70002196C017D107B4F3E5E2F0E080818860D7
:101C8000808380E18A95F1F7DF91CF911F910F91C9
:101C9000FF90EF90089590E0E3E2F0E003C09F5FD3
:101CA000983C19F0808181FDFACF089590E0E3E23D
:101CB000F0E003C09F5F983C19F0808181FFFACF6C
:101CC00008950F931F93CF93DF93EC01E4E2F0E0CC
:101CD00080818D7C808380818C608083E5E2F0E070
:101CE00080818E638083EAE2F0E080818E7E808353
:101CF000EBE2F0E08081816180838AE08A95F1F7F0
:101D0000489B5BC04C9903C08E8180618E83E5E265
:101D1000F0E08081877F80838AE08A95F1F71C99C3
:101D200003C08D8181608D831D9903C08D81846086
:101D30008D83489903C08D8188608D834C9903C041
:101D40008D8182608D83E5E2F0E08081837F886011
:101D500080838AE08A95F1F71C9903C08E818260A6
:101D60008E831D9903C08E8184608E83489903C041
:101D70008E8181608E834C9903C08F8182608F83B6
:101D8000E5E2F0E08081837F80838AE08A95F1F745
:101D90001C9903C08E8180688E831D9903C08E813B
:101DA00080648E83489903C08E8188608E834C99AD
:101DB0003EC18E8180628E833AC11C9B38C1E5E2B0
:101DC000F0E08081877F808380818B7F80830E9489
:101DD0004B0E1C991BC105E210E0F8018081846064
:101DE00080830E94560EF80180818B7F80830E9441
:101DF0004B0E1C9903C08D8181608D831D9903C09A
:101E00008D8184608D83489903C08D8188608D8326
:101E10004C9B02C010E01AC08D8182608D8310E05F
:101E200015C08D8181608D831D9903C08D81846073
:101E30008D83489903C08D8188608D834C9B02C03F
:101E400011E004C08D8182608D8311E0E5E2F0E055
:101E50008081846080830E94560E1C9903C08E810D
:101E600082608E831D9903C08E8184608E83489921
:101E700003C08E8181608E834C9903C08F81826004
:101E80008F83E5E2F0E080818B7F80830E944B0EA0
:101E90001C9903C08E8180688E831D9903C08E813A
:101EA00080648E83489903C08E8188608E834C99AC
:101EB00003C08E8180628E83E5E2F0E080818460E1
:101EC00080830E94560E4C9903C08E8180618E8360
:101ED000E5E2F0E080818B7F80830E944B0E1C99AD
:101EE00002C000E101C000E01D9B0062489B00644D
:101EF0004C9B0068E5E2F0E08081846080830E9472
:101F0000560E1C9B01601D9B0260489B04604C9B0D
:101F10000860113019F48FE7801B8983E5E2F0E057
:101F200080818B7F80830E944B0E1C9902C000E150
:101F300001C000E01D9B0062489B00644C9B006850
:101F4000E5E2F0E08081846080830E94560E1C9B55
:101F500001601D9B0260489B04604C9B086011302F
:101F600019F48FE7801B8A83E5E2F0E080818B7FA4
:101F700080830E944B0E1C9902C000E101C000E06A
:101F80001D9B0062489B00644C9B0068E5E2F0E00A
:101F90008081846080830E94560E1C9B01601D9B83
:101FA0000260489B04604C9B0860113019F4802F3C
:101FB00086958C83E5E2F0E080818B7F80830E94B0
:101FC0004B0E1C9902C000E101C000E01D9B0062A5
:101FD000489B00644C9B0068E5E2F0E080818460EF
:101FE00080830E94560E1C9B01601D9B0260489BD3
:101FF00004604C9B0860113019F4802F86958B8308
:10200000E5E2F0E080818C60808311C005E210E0A1
:10201000F8018081846080830E94560EF8018081DF
:102020008B7F80830E944B0E1C9BFBCEFDCEDF91ED
:10203000CF911F910F910895DC01E4E2F0E08081DF
:10204000817C8083E5E2F0E080818E638083E7E23B
:10205000F0E08081827C8083808182608083E8E2FE
:10206000F0E080818F63808380818D7F8083808199
:102070008260808390E820E1E3E2F0E0822F8A959D
:10208000F1F7808185FF03C011969C9311978081A1
:1020900084FF03C012969C931297808183FF03C034
:1020A00013969C931397808182FF03C014969C9390
:1020B00014979F5F9F3711F711968C9111978E3768
:1020C00019F411961C92119712968C9112978E37D3
:1020D00019F412961C92129713968C9113978E37BF
:1020E00019F413961C92139714968C9114978E37AB
:1020F00019F414961C921497309907C016968C9177
:102100001697816016968C931697199907C01696A4
:102110008C911697826016968C9316974C9907C0EF
:1021200016968C911697846016968C9316974899FC
:1021300006C016968C911697886016968C93089513
:10214000E9E6F0E0808182608083EDE3F0E0808169
:1021500081608083ADE6B1E08BE48C93EFEAF1E03F
:10216000808311978AE58C933197808308951F931C
:10217000CF93DF9380919401982F93500AF4A3C0DA
:1021800020919101809190018D3209F09AC0983090
:1021900009F097C08CE090E0821B9109FC01E856A1
:1021A000FE4FEF0183EC809361018AE5809300018B
:1021B000109232018081807629F0CF010E941202B4
:1021C000982F76C0928110926A018181882331F420
:1021D000EBE6F1E0108292E0319766C0853031F491
:1021E0009093950190E0EAE6F1E05EC08630D1F58B
:1021F0008381813041F488E690E09093930180934D
:10220000920192E12BC0823041F48AE790E09093F2
:1022100093018093920190E221C08330F1F49923DD
:1022200041F487EB90E0909393018093920194E0C6
:1022300015C0913041F48BEB90E090939301809323
:1022400092019AE20BC0923041F485EE90E09093B7
:102250009301809392019AE201C090E080E4809320
:10226000320126C0883021F491E0E7E9F1E01CC09A
:10227000893031F49093970190E0EAE6F1E014C0E0
:102280008A3021F491E0EAE6F1E00EC08B3021F0D3
:1022900090E0EAE6F1E008C08BE480936D01809362
:1022A000AF0190E0EAE6F1E0F0939301E093920150
:1022B0008F81882321F48E81891708F4982F9093B9
:1022C0000101109294018091000184FF57C0109188
:1022D00001011F3F09F452C0193008F05CC0109290
:1022E0000101E1E6F1E0808198E8892780831123EC
:1022F00009F45DC0209192013091930180913201E7
:1023000086FF14C0A2E6B1E080E090E0F901E80F9A
:10231000F91FE491ED9301961817C1F7812F8150B1
:1023200090E00196F901E80FF91F0FC0D901912F34
:10233000E2E6F1E08D9181939150E1F7812F815098
:1023400090E00196F901E80FF91FF0939301E093F3
:102350009201193068F482E691E0612F0E94251203
:10236000612F6C5F6C3040F48FEF8093010104C0EB
:102370008FEF809301016EE16093000194E1E9E247
:10238000F0E080818670D1F49150D9F710929501D8
:1023900010928F0113C0812F885080930101E1E6D4
:1023A000F1E0808198E88927808318E0A3CF82E656
:1023B00091E060E00E94251264E0D6CFDF91CF91DA
:1023C0001F9108951F93CF93DF93DC01162FEA012D
:1023D000888184FF05C0898198E88927898302C0A4
:1023E0008AE58883AE014E5F5F4FFA01212F8D9100
:1023F00081932150E1F7CA01612F0E942512812F9C
:102400008C5F8883DF91CF911F9108954EEA51E050
:102410000E94E21108954CE651E00E94E2110895F5
:10242000A82FB92F80E090E041E050EA609530E0BD
:1024300009C02D9182279795879510F084279527BD
:10244000305EC8F36F5FA8F30895EADF8D939D9324
:102450000895CF93CFB7CF93DF93C395499BE9F707
:10246000499B0BC0499B09C0499B07C0499B05C0BC
:10247000499B03C0499B01C08BC06F93C0919101E0
:10248000DD27C856DE4F2F9365E5499B03C02F918A
:102490006F91E6CF0F931F934F9320E040E15F933E
:1024A00009B1067001FB27F93F9350E03BE039C0CA
:1024B000167040642F77012F5F5F1EC0406819B10E
:1024C00016702F7752501FC0406409B12F770670E5
:1024D000D1F15F5F00C023C0406219B12F77167041
:1024E00091F15F5F00C025C006701027515012F4B3
:1024F0005D5F0000115027952C3F19B1C8F616708A
:102500000127015027952C3FC8F64227499309B16E
:10251000067010274F73115027952C3FA8F646954B
:10252000469519B1167079F00127015027952C3F77
:1025300098F66B5A60F3315009B1B0F600C011E063
:102540001CBB002719C03B503195C31BD04011E084
:102550001CBB0881033C09F10B34F9F020918F0179
:102560001981110F1213EDCF4A81441F093651F121
:102570000D3211F0013E29F7009396013F915F91D2
:102580004F911F910F912F916F91CCB3C0FD65CFEB
:10259000DF91CF91CFBFCF91189520919601222343
:1025A00069F3109194011123E9F53430EAF1309385
:1025B000940120939001109191013BE0311B3093E5
:1025C000910132C000919401013064F50AE54F7029
:1025D00049F43091000134FD28C000930001C1E6A8
:1025E000D1E027C0423049F030916C0134FD1DC06C
:1025F00000936C01CDE6D1E01CC03091AE0136FDF8
:1026000014C00093AE01CFEAD1E013C0052710E05B
:1026100000C000000BB91AC0052710E0221F1DC022
:1026200010E021C04AE502C032ED432FC4E1D0E002
:1026300032E01AB11660599A0BB11AB956E020E887
:1026400065E320FF05270BB9279517951C3FF0F68A
:102650006695B8F7B1F720FF05270BB927951795B1
:102660001C3FD0F62795179517FF052700001C3F44
:102670000BB9B0F629913A9519F7097F1091950198
:10268000110FC651D0400BB911F010938F0111E01A
:102690001CBB02601AB1197F402F497F54E05A9544
:1026A000F1F70BB91AB94BB969CF629FD001739F8B
:1026B000F001829FE00DF11D649FE00DF11D929FDE
:1026C000F00D839FF00D749FF00D659FF00D99271D
:1026D000729FB00DE11DF91F639FB00DE11DF91F41
:1026E000BD01CF011124089597FB092E05260ED0B8
:1026F00057FD04D014D00AD0001C38F450954095F2
:10270000309521953F4F4F4F5F4F0895F6F79095C5
:102710008095709561957F4F8F4F9F4F0895A1E2EF
:102720001A2EAA1BBB1BFD010DC0AA1FBB1FEE1F4B
:10273000FF1FA217B307E407F50720F0A21BB30B96
:10274000E40BF50B661F771F881F991F1A9469F712
:1027500060957095809590959B01AC01BD01CF016E
:062760000895F894FFCF7C
:022766005AFF18
:00000001FF
